:020000020000FC
:1000000005C062C0189573C01895189505E007BB28
:1000100000E008BB01E003BF02E009BF03E005BF49
:1000200000E40BBF06B301FBEEF306B301FBEEF7F2
:1000300000E60ABF0DE001BD789403D014D0A89566
:10004000FCCF30FB7EF0042D083060F0073250F416
:10005000053110F4497F06C00B3110F0466002C034
:1000600042604B7F0895042F0670002341F400E0A6
:1000700008BB3D7FF89466247724789424C0F894D4
:10008000162D272D789441FB3EF0C0983D7FF894C3
:1000900066247724789412C032600EE4011704E0DD
:1000A000020710F0C09A0AC0C09805E101170BE2E0
:1000B000020720F4F89466247724789442FB16F023
:1000C000C29801C0C29A08952FB640FB56F044244E
:1000D00050E052BF52E058BF316052E055BF41601E
:1000E00004C03E7F53E055BF4E7F2FBE18952FB6FC
:1000F00030FB0EF4439431FB1EF4639409F47394C3
:040100002FBE189561
:00000001FF
